:100000000428FF3FFF3FFF3F07300313831299008F
:100010001830831685009F0183128501E830A00007
:100020000330A100A201A301A401A5012508043CFD
:10003000031C2C2805142008A8002108A9009821D9
:1000400005102008A8002108A90098212508043AD5
:1000500003192C28A50A1628A201A5012508313C60
:10006000031C5D280030051A0130D2005208003A06
:10007000031D3B28A20A05146430D400D5012008D2
:10008000D0002108D10082225008A8005108A90000
:10009000982105100A30D400D5012008D00021088D
:1000A000D10082225008A8005108A90098212508F3
:1000B000313A03195D28A50A2E2822081E3C031890
:1000C0006228032922080A3C03186728A728220867
:1000D0000A3C031C6C28742805142008A800210879
:1000E000A900982105102C28A6012608483C031CCD
:1000F000A528A7012708633C031C9F282308053C6B
:1001000003188328912805146430D400D5012008F1
:10011000D0002108D10082225008A8005108A9006F
:100120009821051085142008A8002108A90098210D
:10013000A30A2708633A03199F28A70A7A282608E2
:10014000483A0319A528A60A752885105D29A60135
:100150002608443C031C0229A7012708053C031C70
:10016000D42805140A30D400D5012008D000210875
:10017000D10082225008A8005108A900982105103A
:1001800085142008D0002108D1000530D400D50105
:1001900057225008A8005108A90098212708053ABD
:1001A0000319D428A70AAD28A70127080E3C031C71
:1001B000FC2805140A30D400D5012008D0002108FD
:1001C000D10082225008A8005108A90098210510EA
:1001D00085102008D0002108D1000530D400D501B9
:1001E00057225008A8005108A900982127080E3A64
:1001F0000319FC28A70AD5282608443A031902291E
:10020000A60AA8285D29A7012708033C031C2B295F
:1002100005140A30D400D5012008D0002108D100EF
:1002200082225008A8005108A900982105108514C1
:100230002008D0002108D1000A30D400D50157226F
:100240005008A8005108A90098212708033A03196B
:100250002B29A70A0429A7012708093C031C5329B5
:1002600005140A30D400D5012008D0002108D1009F
:1002700082225008A8005108A90098210510851075
:100280002008D0002108D1000A30D400D50157221F
:100290005008A8005108A90098212708093A031915
:1002A0005329A70A2C29240AD2005208A400520874
:1002B000723C03185C295D290329850105140A3065
:1002C000D400D5012008D0002108D1008222500896
:1002D000A8005108A900982105100A30D400D501C2
:1002E0002008D0002108D10082225008A80051081F
:1002F000A900982105140A30D400D5012008D000A7
:100300002108D10082225008A8005108A900982194
:1003100005102008D0002108D1000A30D400D501F2
:1003200057225008A8005108A90098215D29972953
:10033000E83003138312AA000330AB00AC01AD0117
:100340002808D0002908D100D201D301E830D40018
:100350000330D5000030D6000030D70020225008EE
:10036000AA005108AB005208AC005308AD000030A1
:100370005302031DC52900305202031DC529023056
:100380005102031DC529A33050020318C8291F2A92
:10039000A330D0000230D100D201D3012A08D4000A
:1003A0002B08D5002C08D6002D08D7005008D40201
:1003B0005108031C510FD5025208031C520FD602DC
:1003C0005308031C530FD7025408AA005508AB006A
:1003D0005608AC005708AD000530D0005408AA00FC
:1003E0005508AB005608AC005708AD00500803197B
:1003F000002AAD0CAC0CAB0CAA0CAD13FF3FF729D7
:10040000FF302A05D8002B08D0005008D8042C084B
:10041000D0002D08D1005008D8042D08D000500875
:100420005804D4005408003A03191F2A0130AA02C4
:10043000031CAB02031CAC02031CAD02002A080023
:10044000031383122230DC00D801D901DA01DB0169
:10045000DC030319562A0310DB0CDA0CD90CD80C78
:10046000D30CD20CD10CD00C031C282ADC030319AA
:10047000482A5408D80755080318550FD9075608B5
:100480000318560FDA0757080318570FDB072C2AF3
:100490005408D80755080318550FD90756080318EC
:1004A000560FDA0757080318570FDB070800031326
:1004B0008312DB01DA01D9018030D800D10CD00CD5
:1004C000031C6B2A5408D90755080318550FDA077F
:1004D0000318DB0A0310D01F732A5408DA075508E3
:1004E0000318550FDB07DB0CDA0CD90CD80C031CF6
:1004F0005E2A5B08D3005A08D2005908D100580878
:10050000D000080003138312D801D9011030DC0099
:10051000510DD80DD90D5408D8025508031C550F9C
:10052000D90203189A2A5408D80755080318550FFA
:10053000D9070310D00DD10DDC0B882A0800FF3F2E
:02400E00D43F9D
:00000001FF
